:100000000C94340018950000189500001895000015
:10001000189500001895000018950000189500002C
:10002000189500001895000018950000189500001C
:10003000189500001895000018950000189500000C
:1000400018950000189500001895000018950000FC
:1000500018950000189500001895000018950000EC
:1000600018950000189500008FEF8DBFC0E0E8E103
:100070004E2E88E08EBFD8E0F6E05F2EA89584B7BC
:10008000082E877F84BF88E1992780936000909332
:100090006000EEEFF7E0A0E0B1E088278D933197A4
:1000A000E9F789E18093C40080E08093C50088E18E
:1000B0008093C100662486E08093C2007894259ADC
:1000C0002D98239A2B98219A29980E94DB010E944F
:1000D000AA000E947F02ADE5B1E08C9384E2482F34
:1000E00000915D01041711F00C94A8000E94850294
:1000F000AFE5B1E08C9381E08093600100916001F5
:10010000083218F011F00C9498000E948502A0E6C5
:10011000B1E0AD90BB24ACE0B1E0AA0DBB1D8C9367
:10012000A0E6B1E08C918F5F8C9310F40C947E006C
:1001300040915E0100915F01041711F40C94A60038
:1001400080915F0180935E010E94DB010E94DB00D1
:100150000C94690081E00E949C0281E0A881B98131
:100160008C93A881B9810C91083218F011F00C948D
:10017000D500A881B9818C91D2018C9381E00E9435
:100180009C0280E0D2018C9381E00E949C020E943C
:100190001401249682E00E949802A881B9818C9172
:1001A0008F5F8C9310F40C94B10081E0481A80E0CA
:1001B000580A2296089581E00E949C0281E0A8815D
:1001C000B9818C93A881B9810C91083218F011F093
:1001D0000C940E01A881B9818C91D2018C9381E09D
:1001E0000E949C02AA81BB81AD90BB24ACE0B1E02F
:1001F000AA0DBB1D8C91D2018C9381E00E949C02C0
:100200000E941401249682E00E949802A881B9817C
:100210008C918F5F8C9310F40C94E20081E0481A6B
:1002200080E0580A2296089581E00E949C0281E0B5
:100230000E949C02AE81BF810E947B02AE81BF8181
:100240008C91AA81BB818C9393E0AA81BB810E948F
:10025000A202AA81BB818C918F5F8C93AE81BF81FA
:100260000C9147E00423A881B9810C93A881B9813E
:100270008C918F5F8C93AA81BB818C91D2018C93DE
:1002800081E00E949C02AA81BB818C91D2018C9357
:1002900081E00E949C02A885B9858C91D2018C9343
:1002A00081E00E949C020E945F01269683E00E94EA
:1002B000980282E0481A80E0580A2496089581E066
:1002C0000E949C0281E00E949C0280E0A881B9818A
:1002D0008C93299885E0AA81BB818C93AA81BB81EC
:1002E0004C9101E0041718F011F00C94C201AA819E
:1002F000BB814C91A885B9850C91041711F00C9421
:100300009F01AE81BF818C91D2018C9381E00E94CC
:100310009C020E94C901229681E00E949802AC8151
:10032000BD818C91D2018C9381E00E949C020E943D
:10033000C901229681E00E9498020C94BB01A88119
:10034000B9818C91D2018C9381E00E949C020E9421
:10035000C901229681E00E949802A881B9818C91FE
:10036000D2018C9381E00E949C020E94C9012296D6
:1003700081E00E949802AA81BB810E947B0210F05A
:100380000C946E01299A82E0481A80E0580A24965B
:1003900008950F931F93A881B9810C9118E007FD70
:1003A0002B9A07FF2B98001F2D9A2D981A95B9F7B5
:1003B0000F911F91089581E00E949C0281E0A88125
:1003C000B9818C93A881B9810C91053018F011F096
:1003D0000C947502A881B9818C91D2018C9381E033
:1003E0000E949C028CE0D2018C9381E00E949C02CE
:1003F00081E0D2018C9381E00E949C020E945F0107
:10040000269683E00E949802A881B9818C91D2013E
:100410008C9381E00E949C0289E0D2018C9381E060
:100420000E949C0280E0D2018C9381E00E949C0299
:100430000E945F01269683E00E949802A881B981FC
:100440008C91D2018C9381E00E949C028AE0D201BF
:100450008C9381E00E949C0280915E01D2018C937A
:1004600081E00E949C020E945F01269683E00E9428
:100470009802A881B9818C91D2018C9381E00E946D
:100480009C028BE0D2018C9381E00E949C0287E069
:10049000D2018C9381E00E949C020E945F0126960B
:1004A00083E00E949802A881B9818C91D2018C933B
:1004B00081E00E949C028FE0D2018C9381E00E9437
:1004C0009C0280E0D2018C9381E00E949C020E94F9
:1004D0005F01269683E00E949802A881B9818C91E1
:1004E0008F5F8C9310F40C94E20181E0481A80E055
:1004F000580A229608958C9181508C9308958827EC
:100500000090C00007FE089500C08091C00087FFE2
:10051000FCCF8091C60008953197F1F70895689453
:1005200062F80895E89462F80895481A590A0895FF
:10053000481A8827580A089599275A924A92480ECD
:10054000591E0895903029F08C9186959A95E9F777
:040550008C930895EB
:00000001FF
